:020000040000FA
:020000000528D1
:0800080005288B01850186012A
:1000100087010313831606309F0001308500860197
:10002000FF3087008030810003138312902024204A
:10003000D301332882073334333432342C3406343A
:100040000C34013402340034C830C922CD01D2014D
:100050004D081A200038031930287120CD0A2828AD
:10006000C830C922080000302423D60001302423E0
:10007000D50002302423D4008B23CC01CB01CA014C
:10008000C9012730C8001030C7008522D3013130A4
:100090008C208520A120051856281423D30A03306C
:1000A000D3055308313E8C208520A12007185B28FA
:1000B0001423CE226E28871860281423D3226E289A
:1000C000071965281423D8226E2887196A28142353
:1000D000DD226E28071A6E281423E422C830C922B4
:1000E0004B28D1003230CE00CE0B742879207920F5
:1000F0000800D10E51080F39520486008616861268
:1001000008000130862880308628C03052127120C5
:1001100052161430C92208000C1E8C2899000800C1
:10012000031383160C309900043098000C1203134B
:1001300083128030980003138316981603138312DA
:10014000080053080319AC28013C0319C3285308BD
:10015000023C0319D828ED280430082153307120BF
:10016000693071206E30712065307120203071202F
:1001700057307120613071207630712065307120E8
:100180000330082108000530082153307120613008
:10019000712077307120743071206F3071206F3092
:1001A00071207430712068307120033008210800FC
:1001B000053008215430712072307120693071206F
:1001C000613071206E307120673071206C30712089
:1001D00065307120033008210800023008215330B7
:1001E0007120713071207530712061307120723052
:1001F00071206530712020307120573071206130BE
:10020000712076307120653071200330082108009C
:10021000D70020307120D703031D09290800C2012F
:10022000B321031CEC2103180800072221222F30E0
:10023000C300DF21310D03182F22031C250D0318E5
:100240000800C30B19294218B8210800C20126086A
:100250002704280429042A042B04003C031CB3218E
:10026000031CEC2103180800AC01AD01AE01AF0185
:10027000B001B1013030C300DF212B083102031D72
:1002800053292A083002031D532929082F02031D70
:10029000532928082E02031D532927082D02031D68
:1002A000532926082C02031C6D292608AC022708B6
:1002B000031C270FAD022808031C280FAE022908D3
:1002C000031C290FAF022A08031C2A0FB0022B08B7
:1002D000031C2B0FB10203102014C30B3C2942183E
:1002E000B8210800CE21C201B32103189029303073
:1002F000C300A00DA10DA20DA30DA40DA50D4130AD
:1003000084000F30C400800DF63000070318800011
:100310008403C40B8329C30B79294218B209031043
:100320003030B304B404B504B604B704B804B90457
:10033000BA04BB04BC04BD04BE04BF04C004C104B1
:100340000F30CD00333084004D08460603190800F5
:1003500000080F39031D08000012840ACD0BA429E0
:100360003030C1040800250D031C0800B821080026
:1003700025088039A009A109A209A309A409A50992
:10038000A00FCB29A10FCB29A20FCB29A30FCB29DB
:10039000A40FCB29A50AC20A25070800B201B301A0
:1003A000B401B501B601B701B801B901BA01BB0189
:1003B000BC01BD01BE01BF01C001C1010800A00D0B
:1003C000A10DA20DA30DA40DA50DAC0DAD0DAE0D8F
:1003D000AF0DB00DB10D08002B0D031C0800F1216D
:1003E00008002B088039A609A709A809A909AA09A4
:1003F000AB09A60F042AA70F042AA80F042AA90FE5
:10040000042AAA0F042AAB0AC20A2B0708002008F4
:10041000AC002108AD002208AE002308AF0024087C
:10042000B0002508B10008002C08A0002D08A1008C
:100430002E08A2002F08A3003008A4003108A50050
:100440000800A001A101A201A301A401A5010800C7
:10045000A601A701A801A901AA01AB01080026086D
:10046000A00727080318270FA10728080318280F3B
:10047000A20729080318290FA3072A0803182A0F1F
:10048000A4072B0803182B0FA5070800F121031858
:10049000080025082B06C2002F2203102B08250672
:1004A000C21F803E0800AB01AA01A9010F30A800BD
:1004B0004230A7004030A6000F2108004708A000E6
:1004C0004808A1004908A2004A08A3004B08A4005C
:1004D0004C08A50008002008C7002108C800220811
:1004E000C9002308CA002408CB002508CC00080056
:1004F0002822A6000800AB01AA01A9015608A800FD
:100500005508A7005408A60008005E2253227B224B
:100510002621053078222F2228220A30A600262103
:1005200073308C2023088C2022088C2021088C20FA
:1005300020088C209C2208005E2272218320023039
:1005400008213B0871203C0871203D0871203E08BD
:1005500071203F087120203040020319B12A400861
:10056000B22A303071202E307120410871202030A5
:100570007120483071207A30712003300821080042
:10058000F830CF000000CF0BC22A000000000000AE
:100590000800D000C022D00BCA2A0800282201304F
:1005A000A600EB22080028220A30A600EB22080051
:1005B00028226430A600EB22080028220330A7007E
:1005C000E830A600EB22080028222730A7001030D0
:1005D000A600EB2208005E22871EF02A2F22F22AB4
:1005E0004622F22AF6226B228522080007220C23DB
:1005F000A60A4622A51F042B14222822A60A462258
:10060000A51B082B1422080014220C2346220800E4
:1006100014220C232F22080028220F30A800423079
:10062000A7004030A6000800FF30D80085141E2324
:1006300085101E23D803031D162B08002D30D9006A
:10064000D903031D202B0800031783128D00031705
:1006500083168C130C14031783120C0803138312D4
:100660000800031783128D00031383125A0803171F
:1006700083128C00031783168C130C1555308D00D4
:10068000AA308D008C14031383120D1E452B0D12FE
:10069000080083204E3071206F3071206D30712042
:1006A000693071206E307120613071206C307120A2
:1006B00004300821373071203330712032307120FE
:1006C0003530712034307120080085204130712090
:1006D000643071206A307120753071207330712060
:1006E000743071206530712064307120033008212E
:1006F00021225608A2005508A1005408A00072212A
:100700003D0871203E0871203F087120400871208B
:1007100041087120080005180800142349236523A7
:100720008718902B142321222822A60A871E9A2B91
:100730002F229B2B46227B222F222208D600210823
:10074000D5002008D40065235608DA000030312394
:100750005508DA00013031235408DA000230312321
:06076000C830C922902BF5
:02400E00723FFF
:0642000001001E00260073
:00000001FF
